:1000000000308A002E280000831A0A28A200030E5E
:10001000A3000F288312A200030EA300A3140A0852
:10002000A7008A018313A20E0408A4002008A500DB
:100030002108A60083128B1E1F280B1934282408C0
:1000400084002508A0002608A10027088A00230EA6
:1000500083008312220EA31883160900FF23831640
:10006000900000308A00E628A90B3B280230AA063F
:100070000F30A900AB0A2B08033C03184128AA1132
:10008000AB010B118A111F2883160510831205106E
:100090000830A100000000000000A1175E28A11395
:1000A000AD0C03180514031C051021175E2821133D
:1000B000A10B5028000000000000051484308400CB
:1000C000840B60280000A11B4F28211B57282E29D4
:1000D0002E0B72282808033C031C7028A80A7228DB
:1000E0000130A800AE08031D7D282808013C031834
:1000F0007B28A8037D280430A80001302802FC3E9C
:100100000318C828043EC92807158316071183124F
:100110008710831687108312071083160710831227
:100120000511831605118312C828071183160711BC
:100130008312871483168710831207108316071003
:1001400083120511831605118312C828071183161F
:1001500007118312871083168710831207148316E2
:10016000071083120511831605118312C828071181
:1001700083160711831287108316871083120710C6
:100180008316071083120515831605118312C828DC
:100190004E290A108A100A11820784289528A62859
:1001A000B7282D30840000080319E5280130A1008C
:1001B000A001A00BD928A10BD8284A30A000A00B81
:1001C000DF2800000000800BD628512984011F3051
:1001D00083051F13003083169100073083129900A6
:1001E00083160510831205140130A8002A10AA14E2
:1001F0000F30A900AB01AA1183161F129F161F17FB
:1002000083129F131F141F130030103883169100A0
:10021000831281010730A000A01D1629073081013B
:10022000813084000008C0390F38800064008130BC
:1002300084000008C039200480008B16C0308B0475
:100240000C30A1001F08C33921049F009F149F1880
:1002500027291E08AC002C08AD0044282C08643C5B
:10026000031C3429AA1D37292A15AA1538292A1151
:10027000AA183C2985103D29851483168510831200
:100280002A194429851245298516831685120030BE
:1002900083122A180130AD00AE0068280530AD0089
:0602A000D12820296300B3
:02400E009431EB
:00000001FF
